:020000040800F2
:100000000804002005010008290100082B01000850
:100010002D0100082F010008310100080000000038
:100020000000000000000000000000003301000894
:100030003501000800000000370100083901000800
:100040003B0100083B0100083B0100083B010008A0
:100050003B0100083B0100083B0100083B01000890
:100060003B0100083B0100083B0100083B01000880
:100070003B0100083B0100083B0100083B01000870
:100080003B0100083B0100083B0100083B01000860
:100090003B0100083B0100083B0100083B01000850
:1000A0003B0100083B0100083B0100083B01000840
:1000B0003B0100083B0100083B0100083B01000830
:1000C0003B0100083B0100083B0100083B01000820
:1000D0003B0100083B0100083B0100083B01000810
:1000E0003B0100083B0100083B010008DFF810D08D
:1000F00000F02EF8004800477D020008AFF30080B2
:10010000080400200D488047DFF83400016841F4FE
:10011000E0210160BFF34F8FDFF82800DFF82810DF
:1001200001600A4800477047FEE7FEE7FEE7FEE78A
:10013000FEE7FEE7FEE7FEE7FEE7FEE72701000831
:1001400024ED00E00CED00E00003FA05ED000008EE
:10015000064C074D06E0E06840F0010394E8070014
:1001600098471034AC42F6D3FFF7C4FF14030008DD
:100170003403000870B5194C8320206000256560A9
:10018000A56017486060012000F02EF86168084300
:10019000606014490D60086840F002000860206843
:1001A00040F48030206020688003FCD5206840F057
:1001B0008070206020688001FCD5606820F003001A
:1001C0006060606840F002006060606840F4800039
:1001D0006060086840F01000086070BD00100240C8
:1001E00000841D0000200240012804D0B0F5807F6B
:1001F00003DD012102E000202CE00021802801DD48
:10020000012200E000220A44402801DD012100E033
:1002100000210A44102801DD012100E000210A44E8
:10022000082801DD012100E000210A44042801DD45
:10023000012100E000210A44022801DD012100E043
:1002400000211144012801DD012000E000200844C4
:10025000C01D0001702800D10020704702E008C8CE
:10026000121F08C1002AFAD170477047002001E030
:1002700001C1121F002AFBD170470000C0B0FFF778
:1002800079FF00240AE02146064800F00FF80649ED
:100290000860084600684DF82400641C402CF2DB1E
:1002A00000BFFEE734030008000000202DE9F04FF6
:1002B0004FF040024FF000034FF000044FF00005F4
:1002C000124FDFF84C80934212D030F9039003FBB9
:1002D00001F606F03F0637F906A009FB0AFB5C446D
:1002E00038F906A009FB0AFB5D4403F10103EAE7C4
:1002F0004FEA24444FEA254504FB04F405FB05F5C9
:1003000004EB0500BDE8F00F00BD0000B4030008D9
:1003100034040008B40400080000002004000000B9
:100320005C020008B8040008040000200404000077
:100330006C020008FF0FF60FD90FA80F640F0E0F05
:10034000A70E2F0EA80D130D720CC50B100B530A20
:100350009009C908000837077006AD05F0043B0492
:100360008E03ED025802D1015901F2009C005800A1
:1003700027000A0000000A00270058009C00F20035
:100380005901D1015802ED028E033B04F004AD0582
:10039000700637070008C9089009530A100BC50BEF
:1003A000720C130DA80D2F0EA70E0E0F640FA80FC1
:1003B000D90FF60FFF7F627F8A7D7D7A4276E370E8
:1003C0006E6AF262825A34511D47573CFC30282530
:1003D000F9188C0C000074F307E7D8DA04CFA9C32E
:1003E000E3B8CCAE7EA50E9D92951D8FBE89838508
:1003F00076829E8000809E8076828385BE891D8F56
:1004000092950E9D7EA5CCAEE3B8A9C304CFD8DAF1
:1004100007E774F300008C0CF9182825FC30573CD2
:100420001D473451825AF2626E6AE37042767D7AD9
:100430008A7D627F00008C0CF9182825FC30573C1F
:100440001D473451825AF2626E6AE37042767D7AB9
:100450008A7D627FFF7F627F8A7D7D7A4276E3704C
:100460006E6AF262825A34511D47573CFC3028258F
:10047000F9188C0C000074F307E7D8DA04CFA9C38D
:10048000E3B8CCAE7EA50E9D92951D8FBE89838567
:1004900076829E8000809E8076828385BE891D8FB5
:1004A00092950E9D7EA5CCAEE3B8A9C304CFD8DA51
:0804B00007E774F300000000EF
:04000005080000ED02
:00000001FF
